:030000000219FDE5
:03000B000200AA46
:03002B0002019936
:03005B0002034C51
:0300730002033253
:1000800002030406080C10182030406080040608A3
:100090000C10182030406080A0C000070F1F3F0DDB
:1000A0000D04050D050305030302C2AF306308C24A
:1000B00063857C8AD2AF32C0D0C0E0206227E525BC
:1000C0006002E473E525F4C3334009758A00D26306
:1000D000F57C01D6F58A758B00758D00D262D0E073
:1000E000D0D0D2AF32C3E526334009758A00D2633F
:1000F000F57C01F6F58AC262E526F4603B306803C0
:10010000207213758B00758D00D0E0D0D0C292C2E2
:1001100096C294D2AF32C292C296C294206E0C2084
:1001200066097410D5E0FDE57E4290758B00758DF3
:1001300000D0E0D0D0D2AF32758A00D263757C0097
:10014000C28DD262212B01C4306805206602D29292
:1001500001C4306805206602D29401C430680520CD
:100160006602D29601C4C29330680A2066077411F1
:10017000D5E0FDD29201C4C29530680A20660774AA
:1001800011D5E0FDD29401C4C29730680A206607F9
:100190007411D5E0FDD29601C4C2AFC2AD53E6EFF3
:1001A000C0D0C0E0D2D3D2AFE57D6009E57A60056A
:1001B000757A0041DF757A01C2CEE52A60072074A6
:1001C00049152A410A7800790020742EE580307E96
:1001D00001F430E50278FF53DACF207E0343DA20C2
:1001E000307E0343DA10C2D8C271E580307E01F45C
:1001F00030E50279FFC3E89970CB306103752A18A6
:10020000207403752A18885FD27020740DE52B6066
:1002100004152B411A43DA01C2D82070024178A894
:100220005F206102C2702074367982B70431C3E85E
:1002300094F0400374F0F8E8C4540F28F87984B7B8
:100240000302415FC313C3138721200802C3132095
:100250000A06C3C898F8415F28F8500374FFF8886D
:1002600022E52D54066011E533C313C3132406257C
:1002700022F52250037522FF7882B6045985222484
:10028000A824C3E52495644002A864C3E8956640A9
:1002900002A8668825E569700241C9C3E8AA699A7F
:1002A0005003E8FAE4F9EAC333FBE56BF45B294059
:1002B0000D256AF8E56A6002156A400B41C90AC358
:1002C000E56A9A5002056A78FF8826C26EC3E52661
:1002D00094F84002D26EC3E52594404002D26420D7
:1002E000CF0AD0E0D0D043E610D2AD32C2CF053A2B
:1002F000E57D6009E57B6005757B006128757B0104
:100300007801E52A6005307402152AC3E55F94017F
:1003100040057562006128756300756C00E5622414
:1003200001F56250037562FFD0E0D0D043E610D2F1
:10033000AD32C2AFC0D053E67FC260759100855622
:1003400094855795759104D0D0D2AF32C2AF53E6A1
:10035000EFC2ADC0D0C0E0C0F0D2D3D2AFA8FBA9ED
:10036000FCE57D6007C3E913F9E813F8C2D83071E2
:100370000261BE53DACF207E0343DA10307E03439E
:10038000DA20D271E580307E01F420E502619588A3
:10039000278928A1E553DACF207E0343DA20307E77
:1003A0000343DA10C2D8C271307402A1D17800E5DB
:1003B00080307E01F430E502A1D1885FA1B953DA23
:1003C000CF207E0343DA20307E0343DA10C271204F
:1003D0006102819753DACF207E0343DA10307E0327
:1003E00043DA20C2D8D271885A895BC3E89558F89D
:1003F000E99559F97B007E087A00C3E8948CE9946A
:10040000005005755E008189882178A2E6A82160E8
:1004100055C3E894C8E994005008E4D2E4FB7A0A92
:100420008164C3E89468E994015008E4D2E3FB7A5C
:100430000F8164C3E894D0E994025008E4D2E2FB4F
:100440007A1E8164C3E894A0E994055008E4D2E1DF
:10045000FB7A3C8164C3E89498E994085008E4D29C
:10046000E0FB7A787E00C3E8955CFCE9955DFD30A1
:0F047000E70AECF42401FCEDF43400FD755E00A6
:10047F00C3EC9AED9E5003755E01885C895D855AC9
:10048F0058855B597802A1B9C3E89527F8E99528F3
:10049F00F9307C02A19D307B02A19D307A02A1969A
:1004AF0020750281BAE9FDE8FC81D9E9C313F9E8A7
:1004BF0013F8307902A196E9C313F9E813F83078ED
:1004CF0002A196E9C313FDE813FC206126C3EC9447
:1004DF001CED9402400281F0ED7018C3EC94C850EB
:1004EF00120529C3E529940A5002A1D1755F00D2E4
:1004FF0070A1D1E529600215297888E6F9740020EA
:10050F007F087896B90302789EE624FAFEE4340059
:10051F00FFC3EC9EFCED9FFD9208B90310A208509B
:10052F0007207609D276A13C307602C276A2085017
:10053F0016B9030DECF42401FCEDF43400FD0205B3
:10054F005678007900A19DB90315EC33FCED33FD0E
:10055F00C3EC940AFCED9400FD50047C007D00C3B5
:10056F00EC94FFED9400400678FF7900A19DEC8597
:10057F0075F0A4C5F0A2F733F8790040030205B96E
:10058F0078FF79000205B9E9C313F9E813F8307C55
:10059F000EE9600278FFC3E81338F8E43400F9C3BA
:1005AF00E894FFE99400400278FF885FD2702061E1
:1005BF0002A1D1741FF4552F4BF52FC274EB7002AB
:1005CF00D274752A18307403752A0A306102A1E5B6
:1005DF0020740353DAFE207403752B06D0F0D0E09D
:1005EF00D0D0D2AD43E6103279010206157903025D
:1005FF000615790A020615791E0206157964020698
:10060F001579C80206157817E4D5E0FDD8FAD9F6A2
:10061F00227A147B7802063C7A107B8C02063C7A95
:10062F000D7BB402063C7A0B7BC802063C7902B202
:10063F007DE4C295D5E0FDD294D5E0FDC294D5E01E
:10064F00FDD295D5E0FDD292E576D5E0FDC292744C
:10065F0096D5E0FDD9D9EAF8D5E0FDD8FBDBCEC2BF
:10066F009522C37C007D0075F00005F0EA33FAEBAC
:10067F0033FB50F6EB13FBEA13FAC3E9FFE8FEE88E
:10068F009AF8E99BF95004EFF9EEF8B3EC33FCED6F
:10069F0033FDD5F0DFEDF9ECF822E889F08A20D2AE
:1006AF00D4F8A9F07B0030F70B7BFFF42401F8E9B5
:1006BF00F43400F9E88520F0A4ADF0F8E98520F0D6
:1006CF00A4AFF0FEED2EF974003FFA7C04C3EA13D9
:1006DF00FAE913F9E813F8DCF48BF030F70AE8F4D1
:1006EF002401F8E9F43400F9E889F0C2D4F8A9F04C
:1006FF00227882B6040302075BC3E55F94014003CF
:10070F00020725852224E4F545F546F547F548F51A
:10071F0049C26D02075B7882E6FCD26DE522F523B4
:10072F00783879C7AA40AB41C3EB13FBEA13FAEC55
:10073F00146013C3EB13FBEA13FAEC14146007C332
:10074F00EB13FBEA13FAD1718845894622C3E545BD
:10075F009523F8E5469400F9500CC3E89480E9948A
:10076F00FF401602078CC3E8947FE9940050030200
:10077F00078C787F790002078C788079FF884A8907
:10078F004B22E54A2547F8E54B3548F9854B20E4E0
:10079F00300701F43549FA30E709C3EA94F0401500
:1007AF000207CAC3EA940F50030207CA78FF79FF02
:1007BF007A0F0207CA780079007AF0C3E5249564AE
:1007CF00500AC374019524500B0207E8E54B20E74C
:1007DF000E0207E8E54B30E706884789488A492229
:1007EF0078A4E6FAC3E54A33F8E54B33F9D1A9E922
:1007FF0030E70BC3E89480E994FF40130122C3E86C
:10080F00947FE9940050020122787F7900012278C9
:10081F008079FFE820E715C3E52398F84009C3E87E
:10082F00940140030208497801020849E8F42401C1
:10083F002523F8400302084978FF884C2278A5E663
:10084F00FAA848A9491206A9E930E70CC3E89401B0
:10085F00E994FF401602087EC3E894FFE994005024
:0F086F000302087E78FF790002087E780179FF86
:10087E00E920E715C3E54C98F84009C3E894014018
:10088E00030208A578010208A5E8F42401254CF816
:10089E0040030208A578FF88242278FFC2642069ED
:1008AE003D206A12D264C3E541940A4009C3E5258E
:1008BE0094405002C26479A1E76023E541601F7441
:1008CE00FF8541F0848539F0306A0375F005A4F890
:1008DE00C5F0600278FFC3E895675002A867886686
:1008EE0022C3E54094C8E5419400E5665003142107
:1008FE0000046002F566220209082275E89022784B
:10090E0083E6FFE5E820ECF7A8BDA9BE0573C3E5B5
:10091E007394084052757300E9FA79A0E76044EACF
:10092E007007E574601B020943C3E895746010E517
:10093E00745006600C1402094F0460F902094FE569
:10094E0074F574C39472401B7564C0C39404401351
:10095E00756480C39404400B756440C394044003D3
:10096E0075640075BB0822E5642410500274FFF50F
:10097E00647982B70402219CC3A864E524985002CE
:10098E00A824C3E895664002A86688258826E573E4
:10099E00B4070375BB1022743279A687F0A4C5F094
:1009AE00A2F733F8C3E895644002A864882288242D
:1009BE00882588268867227540007541F022C2AFCF
:1009CE0075C820A8CCA9CDAA3A30CF010A75C82483
:1009DE00D2AFC3EA13FAE913F9E813F8AB3BAC3C18
:1009EE00883B893CC3E89BF8E99C20690A547FF94F
:1009FE0030670241EF414CAD3D8A3DF9EA9D547F8F
:100A0E00FA600478FF79FFAE3EAF3F8B3E8C3FC35A
:100A1E00EC9FFCC3E99CF542A83BA93CC3E89EF8B9
:100A2E00E99FF9C3E54113FBE54013FAE82AF540C7
:100A3E00E93BF54150067540FF7541FF4196AA40CE
:100A4E00AB41AC40AD417E047F02C3EB9404400247
:100A5E001E1FC3EB940840021E1FC3ED13FDEC13C3
:100A6E00FCDEF7C3EA9CFAEB9DFBEF6009C3E913CA
:100A7E00F9E813F8DFF7EA28FAEB39FB8A408B41E5
:100A8E0050067BFF8B408B41C3EB94025002D26722
:100A9E003069047F0341C17892E6FFC3E537948243
:100AAE0040110FC3E53794A040010FC3EF940640E9
:100ABE00027F057E03E541C4540FF9E541C454F0AD
:100ACE00F8E540C4540F28F8C3E89EFAE99400FBF9
:100ADE004009C3EA9402EB940050047A02E4FB61ED
:100AEE003BAA40AB41EBC4FEEAC4540F4EFCC3EA32
:100AFE009CFAEB9400FBC3E813C313F8EA28FAEB55
:100B0E003400FB8A408B41C3EB94024002C26778EB
:100B1E0003EBC4FE7B00EAC4540F4EFAC3EA98FA04
:100B2E004005C3940250027A027892E6FF306002CA
:100B3E00613B855256855357D26043E680C3E49A93
:100B4E00F8E49BF9C3E833F8E933F930670261DC66
:100B5E00E8FAE9FBD3E913FDE813FC88528953C385
:100B6E00EF94036038EF20E00DE82CF8E93DF9EC46
:100B7E00FAEDFB020B97E828F8E939F9C3E82402ED
:100B8E00F8E93400F97AFE7BFFC3EF9403400E8A36
:100B9E00548B55884E894F8C508D518110885489B5
:100BAE00558A4E8B4F8C508D51306920C3E533944E
:100BBE00034019E542A2E713F8E555F42401384045
:100BCE000B20E7087554FFF42401F5558110E8FA5F
:100BDE00D3E813FC8852C3EF94036020EF20E007A4
:100BEE00E82CF8ECFA61FCE8282402F87AFEC3EF50
:100BFE00940340088A54884E8C50811088548A4E33
:100C0E008C50E56BC3335002646BF56B3060028120
:100C1E001A753404D26043E680E52D5406601FA891
:100C2E0040A941C2AF53E67F759100C3E498F59495
:100C3E00E499F595759104D26043E680D2AF22D245
:100C4E0065754400752000306B03752040020C6CF6
:100C5E00D265754400752040306B03752000D2AF0D
:0E0C6E007801206722E52D54066002C265C39E
:100C7C00E5419405401378029405400878039405E7
:100C8C0040027806306902780A206019E544601544
:100C9C0030690AC3E53394034003D53406D2AFD28E
:100CAC006CA14F9122D2AF0000C2AF20672AE54160
:100CBC00C3FB940F40027B0FEB24053073012330F0
:100CCC006A02742820620123F93069027982E58D69
:100CDC0013E58B13C39940B10544E59BF45440B51F
:100CEC002002A13930690A08C3E8940A400108813E
:100CFC0095206502816CC26553E67F759100306763
:100D0C00107594007595FC759104D26043E6808152
:100D1C006CAE40AF41C3EE33FEEF33FF50047EFFA9
:100D2C007FFFC3E49EF594E49FF595A113C3E533CF
:100D3C0094025002816C306502816CD802A14D8105
:100D4C0095C26C53E67F75910085549485559575C5
:100D5C009104854E56854F57D26043E680D2AFE55D
:100D6C002D54066008206A020533020D89306C0D83
:100D7C00206B0A2065071581158102161A2278004E
:100D8C003064053065027801E53775F007A4F9E5A4
:100D9C00F028F5F0E9A2F013A2F113A2F213F53743
:100DAC00C394785003753778C3E53795384008D22B
:100DBC0066C292C296C294306002A1C38550568519
:100DCC005157D26043E68022207D11C2AF75430299
:100DDC00C295D293D2AF759F40020FA3C2AF754399
:100DEC0002C295D297D2AF759F40020FA3307243C7
:100DFC00207D20C2AF754303900177757E20C2968B
:100E0C00C297306204D294C117D295D2AF759F416C
:100E1C00020FA3C2AF754303900177757E20C29277
:100E2C00C293306204D294C137D295D2AF759F432E
:100E3C00020FA3207D17C2AF754303900152C296D7
:100E4C00306202D294D2AF759F41020FA3C2AF752C
:100E5C004303900152C292306202D294D2AF759F7A
:100E6C0043020FA3207D11C2AF754304C293D297E6
:100E7C00D2AF759F43020FA3C2AF754304C297D282
:100E8C0093D2AF759F41020FA3307243207D20C2D5
:100E9C00AF754305900166757E08C294C2953062A9
:100EAC0004D292C1B3D293D2AF759F40020FA3C2AA
:100EBC00AF754305900188757E80C294C2953062EF
:100ECC0004D296C1D3D297D2AF759F40020FA32004
:100EDC007D17C2AF754305900148C294306202D2AF
:100EEC0092D2AF759F40020FA3C2AF75430590011C
:100EFC005CC2943062EBD296D2AF759F40020FA3C6
:100F0C00207D11C2AF754306C297D295D2AF759FA3
:100F1C0041020FA3C2AF754306C293D295D2AF75EF
:100F2C009F43020FA3307242207D20C2AF75430154
:100F3C00900188757E80C292C293306204D296E191
:100F4C004FD297D2AF759F43020FA3C2AF75430127
:100F5C00900166757E08C296C297306204D292E107
:100F6C006FD293D2AF759F41E1A3207D16C2AF75AE
:100F7C00430190015CC292306202D296D2AF759F4F
:100F8C0043E1A3C2AF754301900148C2963062029F
:100F9C00D292D2AF759F41C26622900146757E00F7
:100FAC00C292C296C294C293C297C295C262227870
:100FBC008076090876090876040876FF0876030817
:100FCC0076FF08760A087603087601087601788C95
:100FDC0076010876FF0876FF0876FF0876FF08761C
:100FEC00FF0876030876FF0876FF0876FF0876255B
:100FFC000876D00876280876500876040876FF081C
:10100C00760208760008767A0876FF08760108766C
:10101C0001087600087603227887E6FFC272BF03C8
:10102C0002D2727888E6C394036008C27DE630E190
:10103C0002D27DC27E7889E630E102D27EC3EF9483
:10104C00026008758E01D27302105C758E00C2733B
:10105C00227880E6149000809378A4F67881E614C8
:0F106C009000809378A5F67886E61490008D9317
:10107B0078A6F6789CE67538FF75390CB4020675C0
:10108B0038A075390AB4030675388275390578A30B
:10109B00E61490009A93F569120FA622227896E631
:1010AB00FA7897E6FB7888E6B40305C3EB940EFB5E
:1010BB00307F047A007BFFC3EB9AFCC3948250020F
:1010CB007C827575000575EC8575F0A4C3E5F0940D
:1010DB007D40F222D27F11A81206067A007B007C9B
:1010EB00101205FCE55F2AFA74003BFBDCF37C0471
:1010FB00C3EB13FBEA13FADCF7FEC27F11A822E560
:10110B00EF20E6037520000520903FFFE5201460DB
:10111B0006901FFF1460009304600375EF1253D900
:10112B00BF7581C043FF801205F775EF0243B20311
:10113B00E5B3240420E70DF521E5E320E006852146
:10114B00B343E301120FA67580FF75A40075F13050
:10115B0075D4DF75900375A5FC75F2FC75D501751B
:10116B00A60175E241C292C296C29412060BD293AB
:10117B00D297D2951205F7C293C297C295E4F8F6AF
:10118B00D8FD756B01120FBB1216647898867675B5
:10119B003001C2AF120610120620120606120627E5
:1011AB0012060612062E120606C2AF78FA79FA302C
:1011BB008507D9FBD8F7021C001124115D11A7116B
:1011CB00A878988676120FA675B68075A900757DDE
:1011DB000075885075891275C82475910475D840AF
:1011EB0075A82275B80275E690759B80759D007584
:1011FB00D10E75BC5875BB0875BA1175E880120510
:10120B00F7D2AF12090553DACF207E0343DA203031
:10121B007E0343DA1043DA01C2D8C271120610D230
:10122B00617B037A0CE55E70077A0CDB030211B469
:10123B001206062070030211B4C270E55FC394025C
:10124B0040E1E52F541F856160F561B560D5DAD5B6
:10125B00C26153DACF207E0343DA20307E0343DAB8
:10126B0010C2D8C27178A2E67008D274E52F54E090
:10127B00F52FC27575290012060B307409C3E529C9
:10128B00940A4002D2751205FC7802307402780081
:10129B00C3E55F9840F0C2AF12062012062012067B
:1012AB0020D2AF120610754D007888E6B4030261A8
:1012BB00921205FC788CE6C394015003021392E55D
:1012CB0030C394015003021392207435C3E55F942D
:1012DB00FF5003021392C2AF120635D2AF12060BA8
:1012EB00C3E55F940150EFC2AF1206201206011244
:1012FB000620D2AF12060BC3E55F94FF40E902183C
:10130B000C7F02D27F11A812060BC2AFC27F11A8AD
:10131B00AE5FC3E55F947FD2AF40761205F7C2AFE5
:10132B00120635D2AFDFDC11DFC3EE94057897F6EA
:10133B001206101216A612178F7F0AD27F11A8124F
:10134B00060BC2AFC27F11A8AE5FC3E55F947FD21D
:10135B00AF50E61205F7C2AF1206201206011206B5
:10136B0020D2AFDFD611DFEE24057896F6120610E9
:10137B001216A61217BE12060B11A8C3E55F94FF37
:10138B00500241D402180CC3E55F954D4003855FB5
:10139B004D12060B78017988E7B403027805C3E593
:1013AB005F98400241B4C2AF1206351206351206E1
:1013BB0035D2AF120610753000E4F531F532053138
:1013CB00E531F470390532789AE6781914601278A1
:1013DB003214600D787D14600878FA14600375324E
:1013EB0000C3E53298401715327531B4789986767B
:1013FB00C2AF120635D2AF7898867612060B12065C
:10140B0001E52A700530740221B47801207402784A
:10141B0006C3E55F9840A77888E6C3940360031280
:10142B00060BE52A70030211B4C2AF120FA6E4F546
:10143B0022F523F524F525F526F56AD2AF7885E656
:10144B00C333F568E4F545F546F547F548F549F539
:10145B0073F52CF52DF53775730875BB101205F761
:0F146B00120909E5E820ECFBA8BDA9BEE9700154
:10147A00F8887412090D75730875BB107887E6FE33
:10148A00760211247887EEF6C2AF7564FF1209A5B9
:10149A00852264852265852266D2AF75220175246C
:1014AA000175250175260185636C756D0175B69008
:1014BA0075A903757D017888E6B40307C27D307685
:1014CA0002D27DD268D269753300120F0C120F3125
:1014DA001209C51209CC1209C51209CC1209C50292
:1014EA0014F8C2AF1124D2AF75730075BB08120C81
:1014FA005E120700120D8A120DD41209CC120C4D7D
:10150A00306D0312075C2067031208A830670312C4
:10151A0008EF120D8A120DF91209CC120C5E306D09
:10152A0003120791120D8A120E701209CC120C4D79
:10153A00306D031207EF120D8A120E951209CC12A2
:10154A000C5E306D0312084C120D8A120F0C120930
:10155A00CC120909120C4D120D8A120F3112090D03
:10156A001209CC306935206B3285676485676585D9
:10157A00636C756D0179187A0CC3E53399400FC213
:10158A0069D26A8A358567648567660215A5C3E5E7
:10159A005F940140030214F8021622306A1B206B82
:1015AA0018E535147004C26A81ECF535C3E55F9419
:1015BA000140030214F8021622753600C3E5627868
:1015CA00FA985054307404E52A604D7888E6B403DA
:1015DA0017207D05207607A1F2307602A1F2206B52
:1015EA0007D26B856764A13778F0306B058567642D
:1015FA007820C3E54198500281F8306B1BC26BC258
:10160A007D307602D27DD26A75351285676481F89B
:10161A000536E55F6002C125753600C2AF120FA616
:10162A007887E6FE760211247887EEF6E4F522F54D
:10163A0023F524F525F526F568C26875B68075A9DF
:10164A0000757D00D2AF1205F7120FA6307409C3D8
:10165A00E5369405400221B461C4901A0D7820122F
:10166A0016E8E520B4550CA31216E8E520B4AA033F
:10167A00021686120FBB1216A60216A5901A037836
:10168A00807B0A1216E8A308DBF9901A0F788C7B84
:10169A00181216E8A308DBF9901A2722C2AF12170C
:1016AA0027121701901A00740E1216EDA374041271
:1016BA0016EDA374141216ED901A0378807B0A12A1
:1016CA0016ECA308DBF9901A0F788C7B181216EC2B
:1016DA00A308DBF912173A121718901A2722E49373
:1016EA00F622E6438F01538FFD75EF0275B7A57594
:1016FA00B7F1F0538FFE22438F02438F0175EF0239
:10170A0075B7A575B7F1901A0DF0538FFC22901A90
:10171A000D7455D1ED901A0E74AAD1ED227A307952
:10172A00D07820901A40D1E8E520F709A3DAF72209
:10173A007A3079D0901A40E7D1ED09A3DAF922ABD1
:10174A0077A878BB01027980BB02027981BB0302C8
:10175A007982BB04027984BB05027986BB060279C9
:10176A0092BB07027987BB080279A3BB0902799C5D
:10177A00BB0A027988BB0B027989E8F7227C051239
:10178A000610DCFB22C2AF12062012062712062E12
:10179A0012063512060112062012062712062E120A
:1017AA00063512060112062012062712062E120606
:1017BA0035D2AF22C2AF12063512062E12062712F2
:1017CA00062012060112063512062E1206271206E6
:1017DA002012060112063512062E120627120620BC
:1017EA00D2AF22AE77AF78C2AF120620120620120D
:1017FA000620120601DEF2120635120601DFF8D2C1
:10180A00AF2212178F12178712178775770175780B
:10181A00017579001217ED7C05AD5F120610C3ED54
:10182A00955F70F5C3E55F9401400AC3E55F94FFD5
:10183A0040370218501217491216A612178FC2AF54
:10184A0075EF12121787DCD10579C3E57994035035
:10185A000280C11217870578E5771490009F93F8E4
:0F186A0008C3E57898500280A8121787121787D5
:101879000577C3E577940C50028094120FBB1216BA
:09188900A6C2AF75EF1212178719
:0319FD0002110ACA
:101A00000E0414090904FF03FF0A03010155AA018A
:101A1000FFFFFFFFFF03FFFFFF25D0285004FF0259
:081A2000007AFF01010003FF41
:101A4000234459535F584D32304123202020202019
:101A500023424C48454C492346333930232020202B
:101A60002020202020202020202020202020202076
:101C0000C2AFC2D353D9BF7581C043B20343FF8073
:101C1000752438752503B1C975EF0275E24043F1AB
:101C20002053A4DF75D400D2857DFA780379E67C51
:101C300010752200752300901DD67B0675249875BB
:101C400025013085028142208508D8FBD9F9DCF7CF
:101C500081B4308508D8FBD9F9DCF781B4B189E4C7
:101C600093A3C39A6004DDC381B4DBDBB17B600264
:101C7000812B7B08E493FAA3B15CDBF87A30B15C8A
:101C8000752200752300B17BEAFCEBFDC3ED94FEE9
:101C9000400EB17B8A278B28ED30E0048A828B834B
:101CA000B17B7AC270D8C3ED94FE601350CEBD00F4
:101CB00025EC60097520007521FF0200008100A855
:101CC00027A9280809D804D90281D3B17FEA89AAB3
:101CD000F281C50D81A0C3ED94035049EDA2E092BD
:101CE000007AC5C3E5829400E583941C50902000DF
:101CF00010438F02438F0175B7A575B7F1F030001F
:101D00001FA827A9280809438F01538FFDD804D99C
:101D100002A12089AAE275B7A575B7F1F0A3A10DBC
:101D2000538FFC817C7AC1BD030CE493A3FAB140CC
:101D3000DCF8B138817C817EAA22AB23B15CEBFA5E
:101D4000EA6222752608C3E52313F523E52213F57D
:101D50002250066323A0632201D526EAB1C9B1C986
:101D600075260AEAF4200102D285300102C285B14B
:101D7000C9C3134002C201D526EB22B17FEAFB2082
:101D80008502A17F308502A184752608AE24AF2587
:101D9000C3EF13FFEE13FEB1CDB1C9C3EA13308513
:101DA000024480FA30E703632201C3E52313F523DD
:101DB000E52213F52250066323A0632201D526D91C
:101DC000E52265236523F52222AE24AF250E0FDE22
:101DD000FEDFFCD20122424C48656C693437316326
:041DE000F390060175
:00000001FF
